:020000040800F2
:10500000B81B0020D550000811870008117E000849
:105010000000000000000000000000000000000090
:105020000000000000000000000000006195000882
:105030000000000000000000E18E00089D960008BE
:10504000E7500008E7500008E7500008E750000864
:10505000E75000080D5C0008E7500008E750000822
:1050600000000000E7500008355B0008E75000082A
:10507000E75000088183000800000000E7500008A6
:1050800000000000E75000080000000000000000E1
:10509000E750000800000000E7500008E750000853
:1050A000E7500008E7500008E7500008699F000833
:1050B000E7500008E7500008000000000000000072
:1050C0000348854600F06CFC00480047DDAC000852
:1050D000B81B00200448804704480047FEE7FEE76D
:1050E000FEE7FEE7FEE7FEE739970008C15000083B
:1050F00030B50B46014600202022012409E00D4670
:10510000D5409D4205D31D469540491B25469540F7
:1051100040191546521E002DF1DC30BDF0B51FB40C
:105120000646002082B005464024019100901BE015
:10513000019922460F46304600F06EFB049A059B0B
:10514000801A994110D310461946224600F054FBAC
:10515000361A8F410197224601200021009F00F05E
:105160004BFB38184D4100902046641E0028DFDCC0
:10517000019B00982946324607B0F0BD03460B4319
:105180009B0703D009E008C9121F08C0042AFAD2FD
:1051900003E00B780370401C491C521EF9D2704783
:1051A000D2B201E00270401C491EFBD270470022BF
:1051B000F6E710B513460A4604461946FFF7F0FF16
:1051C000204610BD30B504460020034600E05B1CBD
:1051D000934203D2E05CCD5C401BF8D030BDF8B503
:1051E00002464A40D40F42004B0052085B089A42E4
:1051F00002D20246084611464A0023D0C30D4A0097
:10520000DDB2120EAD1A202D35DA49020126490A07
:10521000F6058A19002C00D0524220214F1B11465E
:10522000B9402A411018C20D9A4221D0002C17D043
:10523000012D08DCDA05801AD20F8019D207DBB203
:1052400000F016FBF8BDDA05801A012340001B06AA
:10525000C01880185A428018CA0F1043490007E04E
:105260004908C2071143DA05801A801940088018DE
:1052700000F0F6FAF8BD61000122511A001BF7E7B1
:105280000122D2075140AAE70122D2075040A6E7E7
:1052900070B502464A40D50F40004A00ED0740086D
:1052A0005208002814D0002A12D0C40DD30D410298
:1052B0000120C0055202490A520AE41A09181218BC
:1052C0007D34914201D3641C00E04900002C01DAD6
:1052D000002070BD0023914201D3891A0343400886
:1052E00049000028F7D100290AD0914202D10121BA
:1052F000C90705E0914201D2012101E00121C94322
:10530000E005C018401900F0ABFA70BD420005D0AE
:105310004200120E52428A4201DB00207047C9054A
:1053200008187047F0B507460846584087B0C00FC8
:10533000049048000E46590040084908BC1A8841AC
:1053400005D2384631461E4617460B4602465800DF
:10535000400810434CD0300D039040055900400DDB
:10536000490D0590401A0290402872DA1803012175
:10537000000B09050843019004980092002805D00D
:1053800001995242002088410092019002984021E8
:105390000A1A0199009800F02FFA05460C466B4650
:1053A00007CB00F04AFAC0197141039A0E0D002391
:1053B000D71756401A467A40164344D0049A002A1A
:1053C0002DD0029A012A039A15DC1205C01A9141C8
:1053D00001263605001C7141D20F059ED2070093AD
:1053E000019202962A46234600F088FA07B0F0BDE3
:1053F00038463146FAE71605224A0F46B218C01A57
:10540000B74101210905001C4F4100187F41114699
:1054100018187941E20F10436D19644113E0E20757
:105420006D0815436408C2071443039A0126120548
:10543000C01A91413605001C7141CE074008304327
:105440004908C01851412A46234600F04AFACDE7E0
:10545000FFE7049801224000C117121A00238B4174
:1054600004983146C417381AA141EEE730B401243C
:10547000E407634030BC55E730B40124E4076140E1
:1054800030BC4FE70000E0FFF0B51FB488B00B99C7
:105490000998002448400999C00F4900490809911A
:1054A000C0070B990090490049080B910999089889
:1054B000A64608431CD00B990A98084318D00998AF
:1054C00001244000420D4800410D099824050003C5
:1054D000000B204309900B980003000B20430B9016
:1054E00050181C494018002201901446104605E04F
:1054F000002001460DB0F0BD032801DA034600E0AC
:1055000003239C46C11A0AAE0AE05F0008ADED5BBA
:105510004F00F75B7D430027AA187C41491C5B1EA6
:105520006145F2DD410004AB5A522104120C0A43DA
:10553000240C401C0828DFDB01980290009970467B
:1055400001910090059B049A0799069800F0D6F9FE
:10555000D0E700000DFCFFFFF0B50C465C4085B0C5
:10556000E40FE40703944C000026640859009446B5
:10557000490802460296224321D062460A431ED0C1
:105580006200570D4A000E032303550D0124024605
:105590002C492405781B1B0B360B4018234326434C
:1055A000614600901C46501AB44103D30098401C39
:1055B000009002E0921800985B41002803DA002076
:1055C000014605B0F0BD00200121090507468646C9
:1055D00011E064461D46141BB54106D36546521BB7
:1055E000B341744607430C43A646CD07400849081B
:1055F000284392185B4105460D43EAD110461843F3
:1056000013D06046194650407140084306D06046AA
:10561000101AB34106D20122002306E00022012322
:10562000DB0702E00122D2435310009874460105C3
:10563000381C6141029C039D0019694100F051F939
:10564000BFE70000FD030000C217C10F504010B5B6
:105650004018CA079623002100F00AF910BD10B5C2
:1056600000229623114600F003F910BD0EB5C217B3
:10567000C10F5040CA0740180021054B0293019208
:1056800000910A460B4600F039F903B000BD000056
:10569000330400000EB505490291002100910A462D
:1056A0000B46019100F02AF903B000BD330400005D
:1056B000410040020122400AD205090E80187F29CC
:1056C00001DA00207047962903DC9622511AC8405F
:1056D000704796398840704770B5CD0F4A0009036E
:1056E0000123090B1B0519430B4BED070024520D39
:1056F0009A4201DA002070BD074B34339A4203DC32
:105700009A1A00F089F802E00449511888402C43A5
:10571000F1D0404270BD0000FF030000CDFBFFFF51
:105720004A0009030123090B1B051943094B10B556
:10573000520D9A4201DA002010BD064B34339A42D2
:1057400003DC9A1A00F068F810BD0349511888402C
:1057500010BD0000FF030000CDFBFFFFC20FD2070A
:10576000400040080BD0C10D0723DB01C9184002DF
:105770000905400A1143C208400711437047002041
:105780000146704710B5002904DB0124E4074042BC
:105790008C412146002B04DB1C460123DB075242CF
:1057A000A341994200D1904210BD0000CB0FDB070E
:1057B000490010B5490802460A4307D00A0D0724DC
:1057C0000903E401090B121B002A01DC002010BDB3
:1057D000C900440F0C43C100E018D205801800F046
:1057E0003FF810BD0122D207002800DB101A002963
:1057F00000DB511A8142704710B5202A04DB0146B4
:10580000203A9140002010BD914020239C1A03466D
:10581000E3401943904010BD10B5202A04DB084630
:10582000203AD040002110BD0B46D340D040202468
:10583000A21A91400843194610BD10B5202A06DB74
:10584000CB170846203A1041C1170B4306E00B4620
:105850001341D0402024A21A91400843194610BD9C
:10586000002904DA401C490001D14008400070477B
:1058700070B40024050C05D11024000402D10029C5
:1058800021D01124050E01D100020834050F01D1E9
:105890000001241D850F01D18000A41C002801DB1C
:1058A0004000641C002908D020252E1B0D46F54021
:1058B000A14000D001212943084301061B1B000A17
:1058C000DB1D02D5002070BC7047DB05181880185E
:1058D0000029F8DA401C4900F5D170BC40084000AE
:1058E000704710B5002B08DA0024401C6141921863
:1058F0005B411A4301D14008400010BDF0B51FB410
:1059000082B005460C0003D0084604F0E1FB02E03B
:1059100004F0DEFB20300246009021462846FFF7C7
:105920006BFF049B059A04460F4618431143084336
:1059300014D0184610431BD0009840210A1A18466C
:105940000599FFF769FF05460E46009A05990498E8
:10595000FFF752FF084305D0012004E020463946F6
:1059600007B0F0BD0020C11705430E432C43374359
:1059700000990E986305401A7905E40A00220C4349
:10598000FD0A0A3002D500200146E9E70105101999
:1059900069410C9C0D9D00196941FFF7A2FFDFE7EB
:1059A000064C0125064E05E0E36807CC2B430C3C72
:1059B00098471034B442F7D3FFF786FB5CB0000879
:1059C0007CB0000870B58C180578401C6B075B0F25
:1059D00001D10378401C2A1106D10278401C03E053
:1059E00006780E70401C491C5B1EF9D12B0705D4AC
:1059F0000023521E0DD40B70491CFAE70378401C9B
:105A0000CB1A921C03E01D780D70491C5B1C521EC2
:105A1000F9D5A142D8D3002070BD000038B50446A6
:105A2000064805490068FFF763FB604300E0401E3D
:105A300000900028FBD138BD40420F0070010020CB
:105A4000F8B50446006881688907890F012902D1E9
:105A50000168C90722D18168114A10261140012529
:105A600000290ED18168294381600120FFF7D6FF0C
:105A700001F006F807460CE001F002F8C01B0A2806
:105A800007D9606D30436065A06D2843A065012093
:105A9000F8BD20680068C043C007EDD10020F8BD04
:105AA00017000080F8B51848808F00282AD0174CBE
:105AB0000125E16AED051648A94201DB022100E05B
:105AC0000021017000F0CAF90126F6020527A08224
:105AD0003F070FE00F4801F0EDF980B2A083E18BA2
:105AE000421A032A01DC814204D9E0833146384658
:105AF00000F0B0F9E06AA842ECDA012231463846FB
:105B000000F0B7FFF8BD0000A40D00202401002024
:105B10006C000020C015002010B500231A4603E0D9
:105B2000845CE3189BB2521C8A42F9D3D84380B2FA
:105B300010BD000010B5034800F05EFD024800F003
:105B40005BFD10BD541700200C17002030B5446CCD
:105B50001C252C400125A540046C65600468636029
:105B60008368102B036803D099600068C26030BD61
:105B70009A600068C16030BD1449012048720A462D
:105B800002205E32507203203C3A507204200E3ADA
:105B900050720F480D4B0078087022310870203188
:105BA00008770C495A1C0878587149789971233341
:105BB00018715971203318775977107551751A4635
:105BC0001E3210755175107651767047A411002061
:105BD000260100204C01002010B503F097FC202086
:105BE00003F052FD012004F0D3FD002003F04CFD32
:105BF000044804F071FC044804F020FF002004F085
:105C000055FF10BDE800002083800000F8B503F0C8
:105C100049FD05200121000700F01EFF0025144C5E
:105C2000002800D06560134E0221304600F014FFBA
:105C3000002815D1012020700F48808F00280ED039
:105C40000127BF0200223946304600F012FF0A2029
:105C500004F0F4FB01223946304600F00AFF65608B
:105C6000012000F031FE022000F02EFEF8BD000001
:105C70005C01002000040050A40D002070470000CB
:105C800010B5084900224A6107494B684C15234367
:105C90004B604B68082423434B60C009C00102607D
:105CA00010BD00009C170020002002407FB5002599
:105CB0000C460646039500F0D7FDE009029003A9C3
:105CC00001960095684600F067FD002804D000F0BA
:105CD0009FFD002004B070BD00F09AFD0120F9E79F
:105CE00010B5002302E0C45CCC545B1C9342FAD391
:105CF00010BD000010B5214A00219069C30520485D
:105D000004D54169022319434161911593699B05AB
:105D100005D5436901242343436163021943936911
:105D20005B0505D54369082423434361E301194317
:105D300093691B0505D5436904242343436163022A
:105D4000194393699B0405D5436910242343436198
:105D50006302194393699B0304D5446920231C43C0
:105D6000446119439369DB0305D543694024234308
:105D70004361A0020143916110BD00000020024078
:105D80009C17002070B5054600F07AFE0646184CB8
:105D90000AE0681C08D0002D04D000F071FE801BC2
:105DA000A84201D9032070BDA069C007F1D1A06944
:105DB000800701D50220A061A069C00511D4A069A7
:105DC00080050ED4A06940050BD4A069000508D455
:105DD000A069800405D4A069800302D4A069C0032F
:105DE00003D5FFF787FF012070BD002070BD0000C4
:105DF00000200240F8B51746002605460C4600F084
:105E000033FD09E029460220226800F00FFD00283A
:105E100004D1241D2D1D361DBE42F3D300F0F8FC25
:105E2000BE4201D20020F8BD0120F8BD10B50849DE
:105E300002460020054B497905E044001C5B944272
:105E400003D0401CC0B28842F7D310BD48130020D5
:105E50005800002010B500F004FE10BD10B5094830
:105E600001F028F880B2FFF715FC074A074BFFF74F
:105E70000BFB0022064BFFF76FFBFFF751FC80B2D4
:105E800010BD0000C0150020F853E3A59B843E40E0
:105E900000408F4070B50024204602F0B9FF47490A
:105EA0004748A200641CE4B28150142CF9D346493F
:105EB00044480A7902754979417544490A7802765D
:105EC000497841763F490520133148720A2004F091
:105ED000A5FD7D20400104F0BBFD3A4900221331AD
:105EE0000C2004F085FE00210C2004F093FE3848BD
:105EF00000F0E0FF344C0125223C2085AD0309E091
:105F0000334800F0D7FF80B22085E18EFF392D396C
:105F1000884206DBE18E80B28842F1D3491988427B
:105F2000EED8022004F0CAFD002002F071FF294DD6
:105F300000210F2004F0F2FC28422064F8D0206CED
:105F4000411C38D0400435D58122D20100210F20D8
:105F500004F023FE0021102004F0E0FC4106194863
:105F6000490E0022C73004F00FFD164DC735687A80
:105F700005281FD102221549681DFFF723F90028C3
:105F800018D11148AE7C66710422691C3630FFF7C7
:105F9000F5F829461331084672000D466930FFF7BF
:105FA000EDF860792946420005484838FFF7E6F8E1
:105FB0000320207070BD04F0E9F80000FFFF01002D
:105FC000A8130020051200207A0000204C010020B8
:105FD000C015002000D0272410B5084800F096FA1C
:105FE0000A21064800F032FA044800F01DF9800545
:105FF00003D5024800F01AF980B210BD64150020E4
:10600000F8B52F4D00220121284600F032FDFFF7A0
:10601000E3FFFFF724FB2B4E3146FFF739F92A4CFB
:106020000122A0601146284600F023FD2749A06800
:10603000002588423EDB2078254F002815D02570AA
:10604000FFF7CAFFFFF70BFB3146FFF721F9A0600E
:10605000FFF784FB00223B46FFF708FA00221D4BA6
:10606000FFF712FAFFF7A2FB6060A068FFF776FB6C
:1060700000223B46FFF7FAF9174A184BFFF704FADC
:1060800006460F466068FFF769FB134A144B5242FD
:10609000FFF7FAF932463B46FFF744F9FFF786FB74
:1060A00010496060884201DD616004E0FF21C9059C
:1060B000C84200D365606068FFF7FAFAC0B2F8BD65
:1060C0000004005000401B443000002000006040ED
:1060D00000000C4000E064403333333333B33040CE
:1060E000CCCCEC3F0000C842F8B50546044640352C
:1060F000287C0026012808D00120287420688168A7
:106100008907890F01290ED101E00220F8BD01683D
:10611000C90708D0606D2021084360650126002072
:1061200028743046F8BD616DFF220132914302228E
:1061300011436165C1688907890F0091C1688908A9
:106140008900C1602068816892071143816000F076
:1061500097FC07460EE000F093FCC01B0A2809D903
:10616000606D022188431021084360650020287477
:106170000120F8BD206880680028ECDB2068C16839
:10618000009A1143C160606D80088000401C60650A
:10619000C5E70000F8B506460D464036317C0129BA
:1061A0000DD00121317401688A68520709D5416D0B
:1061B000202211434165002030740120F8BD0220E7
:1061C000F8BD174B6A68D80547109A42154C8A6A81
:1061D0002B6812D05B035B0B1A438A622968490360
:1061E00005D5A1680143A1600A20FFF717FC2868C4
:1061F000800312D5A06838430EE05B035B0B9A4323
:106200008A622968490302D5A1688143A160286890
:10621000800302D5A068B843A06000203074F8BDA8
:106220000110000000270140406D70470068006CBD
:106230007047000070B5040006D0606D264600254A
:106240004036002802D006E0012070BDA5653574F7
:10625000204600F0D3F8606DC00603D4216888683A
:10626000400705D5606D1021084360653574EBE784
:10627000606DFF22013290430222104360658868FE
:106280008207920F5B48012A02D10A68D2072BD1FC
:10629000032362689B079A4205D05B429A4202D070
:1062A0005B009A4209D10A69920092080A6121684A
:1062B0000A6963681A430A610CE00A69920092084D
:1062C0000A6181680F22920491438160816862684B
:1062D000114381602168CA6818239A43CA60216803
:1062E000CA68A3681A43CA608168012252069143B2
:1062F00081608168A28E52061143816020688168A6
:10630000C90004D48168012212071143816020680A
:10631000C168394A1140C1602069E168022825D06E
:1063200000200143204620300278037B52035B00AB
:106330001A431143226B1143A26992031143E2698C
:10634000D20311432268D3681943D160616A0A46B7
:10635000FF3AC23A05D0A26A11432268D3681943B2
:10636000D16042780121012A02D00BE00420D8E755
:106370000078002823D0606D202210436065A06D56
:106380000843A065E06B012820681FD00169C90798
:1063900003D0016949084900016120684169C908C1
:1063A000C900416120684169A26B11434161A56543
:1063B000606D80088000401C6065002070BD206812
:1063C000C26801231B041A43C260DBE70269FF2392
:1063D0009B009A43026120680269236CA66C1A43F1
:1063E000636C33431A430261206802690A43026105
:1063F000D3E70000002701401902FEFF10B586B068
:10640000044614216846FEF7D2FE0E4920688842F1
:1064100016D10D48416B421511434163C16A0122F7
:106420001143C162C06A6946104005900220009085
:1064300003200190002002900520000700F050FA90
:1064400006B010BD0024014000100240F8B504461B
:106450004069254640350E4608280BD02068C068A4
:10646000C00709D0606D20210843606500202874B2
:106470000120F8BD082700E00C2700F001FB009088
:1064800011E0701C0FD0002E05D000F0F9FA009931
:10649000401AB04207D9606D0421084360650020AE
:1064A00028740320F8BD206800683842E9D0606D88
:1064B00001214902084360652068C16809058A0F07
:1064C0000C21002A1BD12022125D002A17D102685C
:1064D000120714D5826853070122002B08DB43689A
:1064E0008B434360606D130298431043606506E080
:1064F000606D202318436065A06D1043A065A069FE
:10650000002801D1206801600020F8BD70B5044664
:10651000216800208968490721D425464035297C17
:1065200001291CD001212974E169012904D02046E8
:10653000FFF786FA002811D1616D0A4A1140FF2247
:106540000132114361650021A165297422681C2173
:10655000116021688A6804231A438A6070BD022092
:1065600070BD0000FEF1FFFF30B5014620314A79D1
:106570000023022A04D00422C2630B71012030BD23
:10658000026814680E25AC4314600268146864083D
:1065900064001460446C1C22144001221546006CF7
:1065A000A54045604A7118460B7130BD70B5002496
:1065B000014620314A79022A03D00421C163012413
:1065C00018E0026813680E25AB4313600268136875
:1065D0005B085B001360436C1C22134001221546CC
:1065E0009D40036C5D604A7100220A71816B002935
:1065F00000D08847204670BDF0B4016C0D6801687A
:106600000C68466C1C2304221E401746B7402F42DC
:106610000ED067070CD50C68A40602D40C6894430E
:106620000C60416C19408A40016C4A60016B1AE0B1
:106630000227B74002462F402032002F17D0A7076D
:1066400015D50C68A40605D40C680A25AC430C606B
:1066500001215171446C02211C40036CA14059601E
:1066600000211171C16A002918D0F0BC0847082721
:10667000B7402F4212D0240710D50C680E25AC432A
:106680000C60446C01211C400B46A340046C636009
:10669000C163517100211171416BE4E7F0BC704797
:1066A00070B504003CD01F48256814212818FEF757
:1066B0001FFD800060641C482064022120462030B9
:1066C0000246417129681948E3680140A06866697B
:1066D0001843236933431843A3691843E3691843F4
:1066E000236A1843084328600121A068890388426F
:1066F00010D00D488030836A656C1C210D400F2638
:10670000AE40B3438362656C63680D40816AAB4001
:106710000B4383620020E06301215171107170BD51
:10672000012070BDF8FFFDBF000002400F80FFFF99
:10673000F8B504468C46203001790025012909D09E
:106740000126067141790027012905D0077102252C
:106750002846F8BD0220F8BD02214171E763206898
:10676000016849084900016061462046FFF7EEF9DB
:10677000206B00282068016801D00E2205E0042269
:1067800091430160206801680A221143016020687A
:10679000016831430160DBE7F8B51A4E0546307CED
:1067A0000F46012807D0012030741748FFF7EAFA96
:1067B000010002D021E00220F8BD0020C043386073
:1067C0006C6814E02046FFF75BFA0F48FFF7DAFA2F
:1067D00001460E48426808239A43426042684315C6
:1067E0009A434260002901D03C6006E08034A868EA
:1067F0006A68C0018018A042E4D8002030740846BE
:10680000F8BD00009C17002050C30000002002408B
:106810000548416802221143416041680122114349
:10682000416000207047000000200240F8B50C4C89
:106830001646207C0F46012808D001202074094804
:10684000FFF7A0FA0025002802D006E00220F8BDDC
:1068500065613E600348FFF795FA2574F8BD0000B6
:106860009C17002050C3000011484168C9070BD095
:10687000EFF3108172B60F4AC2600F4AC26081F313
:1068800010884168C9070ED1416889070DD5EFF31B
:10689000108172B6094A0261094A026181F31088C7
:1068A0004068800701D50120704700207047000034
:1068B00000200240EFCDAB8905040302BFAE9D8CE2
:1068C000161514137047000010B504494A690242B6
:1068D00002D04861FFF7F6FF10BD00000004014040
:1068E000FCB500230124A2E027462A469F403A40F7
:1068F0006FD04D68012D05D0022D03D0112D01D090
:10690000122D16D185680326AC465D00AE46AE401A
:106910006546B543AC46CE687546AE4065462E43E7
:10692000866046680D79BE43ED06ED0F9D40354308
:106930004560C6685F000325BD40AE46AE433546A0
:106940008E68BE402E43C6604E68022E01D0122EC5
:1069500014D1DE08B60036180196366A5D07B446D3
:10696000EE0E0F25B54000966646AE43B4460D695F
:10697000009EB54066462E43019D2E620668754610
:10698000AE430D79AD07AD0FBD40354305604D6891
:10699000ED004BD5294D6E6B26436E639E08284D46
:1069A000B6007519AC46AD689E07360F0F27B74085
:1069B000BD4305273F07B84201D1002715E0214F0D
:1069C000B84201D1012710E01F4FB84202D102277F
:1069D0000BE02BE01D4FB84201D1032705E01C4F0F
:1069E000B84201D1052700E00627B7402F4365468E
:1069F000AF60184D2E684F689643FF0300D51643CD
:106A00002E606E684F689643BF0300D516436E60D4
:106A1000AE684F689643FF0200D51643AE60EE683D
:106A20004F689643BF0200D51643EE605B1C0A68B0
:106A30001546DA4000D057E7FCBD000000100240C8
:106A4000000001400004005000080050000C0050FD
:106A5000001C0050000401400069084000D00120E3
:106A60007047426913460B401B0491430B438361FB
:106A70007047002A01D08161704781627047000031
:106A80000148806870470000640100200248816866
:106A900002788918816070476401002010B50848A9
:106AA00000240168402211430160204600F00AF8EA
:106AB000002801D0012401E000F046FA204610BD74
:106AC0000020024070B504460D4D7D202978C0009D
:106AD000FEF70EFB01460B480068FEF709FB00F0CD
:106AE0002FFF002809D1042C07D200222146401E86
:106AF00000F052FA00206C6070BD012070BD0000F3
:106B0000640100207001002070477047F8B502F062
:106B1000C9FD624C0120E070208AFEF7A0FD01460D
:106B20007F20C005FEF7B4FB5D4D06462968FEF7E1
:106B300056FB28600120E56AC005854201DA284637
:106B400007E030460121FEF7E1FB2946FEF79CFBFA
:106B5000E062FF21C9050025C84200D3E5626078E4
:106B600000280BD102214F48FFF776FF02004E4963
:106B70004E4817D00022FFF77CFF256302214948C9
:106B8000FFF76AFF4A4E002855D02563B08AFEF70A
:106B900066FD434F3968FEF725FE5FD24549012067
:106BA00008705DE00122D1034048FFF762FF208AB0
:106BB000FEF755FD01467F20C005FEF769FB216BFE
:106BC000FEF70DFB3C4920638842D7DD384801279A
:106BD000F926403000900A213046FEF789FA002954
:106BE00003D131493148FFF735F902212D48FFF72C
:106BF00033FF002801D0002701E0002F12D102212D
:106C00002848FFF729FF00280CD104F039F9009932
:106C10000120888004F092F9642003F00FFC2849D9
:106C20002648C8600A2003F009FC3046761EF6B2FA
:106C30000028D0D1A2E7208AFEF711FD01467F206F
:106C4000C005FEF725FB216BFEF7C9FA1D4920633D
:106C500088429BDB1A491948C86097E715480570B8
:106C6000708F401EFEF7F0FC3968FEF7BBFD06D8BA
:106C70002079002803D014490120087001E012484F
:106C80000570708FFEF7EBFC3968FEF7ABFD04D2A0
:106C90002079002801D004F0B5F8F8BD24010020C7
:106CA000600100200004005000800000000000503F
:106CB000A40D00205E000020000040400400FA0502
:106CC00000ED00E00000A0406E000020704770B5AD
:106CD000040010D0022025462035A873204601F07C
:106CE00057FBA87B032805D0204600F0B9F8002008
:106CF000A873687370BD012070BD7047704710B5F0
:106D0000044600680168C943C90708D18168C943BE
:106D1000C90704D1012141602046FFF7F7FE206832
:106D20000168C943890708D48168C943890704D425
:106D3000022141602046FFF7E7FE20680168C94351
:106D4000490708D48168C943490704D40421416034
:106D5000204600F0F7F820680168C943090708D405
:106D60008168C943090704D4082141602046FFF720
:106D7000ADFF20680168C943C90608D48168C943CA
:106D8000C90604D4102141602046FFF7BEFE2068EA
:106D90000168C943890608D48168C943890604D4B7
:106DA000202141602046FFF7A9FF20680168C94300
:106DB000490608D48168C943490604D4402141608A
:106DC0002046FFF79AFF10BDF8B5040005D0254610
:106DD0002035A87B002802D006E00120F8BD002065
:106DE0006873204600F04EF80220A8732068C2683D
:106DF00084466368012B01D10620824316486169ED
:106E0000814202D0072040038243002B01D1D820C9
:106E100082431248A668024018463043676A266AD1
:106E20003E433043A66A30431043002B02D0012B6F
:106E300004D005E02369E2691A4300E0E2681043E8
:106E4000054A914202D0A269114308436146C860D5
:106E50000120A8730020F8BDFFFF0000F8F119FF22
:106E600010B500680549884207D10548816B490083
:106E7000490881630D2000F073F810BD007C0040CC
:106E80000010024010B50068084988420CD108483B
:106E9000816BC20411438163002201210D2000F0A7
:106EA0007BF80D2000F06CF810BD0000007C004065
:106EB000001002400068C06970470000F8B5044641
:106EC0000220254620351746A8731D480268C304D2
:106ED0001A4302602068C2689B121A43C26020688D
:106EE0000269012632430261226810205060206846
:106EF00081611021204601F0BBFA03281FD02168D0
:106F000008204860206847610821204601F0B0FA57
:106F1000032814D0204601F03BFAA87B03280ED0AA
:106F200020688168314381602068016931430161D3
:106F300020680169042211430161AE730020F8BD8D
:106F400000040140704700000448416B01221143D6
:106F50004163816B0204114381637047001002405A
:106F6000002809DBC106C90E0120884003490860DA
:106F7000BFF34F8FBFF36F8F7047000080E100E0D9
:106F8000002805DBC106C90E0120884001490860C0
:106F90007047000000E100E010B503F0D5F810BD27
:106FA00002494A6882434A6070470000007000400E
:106FB000024801688215114301607047007000406B
:106FC00002494A6802434A6070470000007000406E
:106FD0000548016802221143016004480169042246
:106FE0001143016130BF70470070004000ED00E0C8
:106FF000F0B5154A1368154D54152D6A2340ED0759
:10700000ED0F002B04D0002D02D01668A6431660A9
:107010001668B608B600064316600D4807690426D0
:107020003743076101290DD040BF20BF20BF016950
:10703000B1430161002B04D0002D02D01068204321
:107040001060F0BD30BFF2E700700040000001406A
:1070500000ED00E0F8B5044600780027534D8006A7
:1070600071D5524E403EB06BC00004D4B06BA90540
:107070000843B06301274E480168C90511D401686F
:10708000821511430160FFF7FBFC009005E0FFF75C
:10709000F7FC0099401A642837D845480068C005B5
:1070A000F5D532680321090560680A400140914224
:1070B00008D08103890F032904D13168890301D5E0
:1070C0000120F8BD2A69032109040A4022D00840A2
:1070D00090421FD0207880061CD528692A698843F1
:1070E0000121C9040A432A612A698A432A61286165
:1070F000C0050FD5FFF7C4FC009008E0FFF7C0FC07
:107100000099411A2B48814201D90320F8BD286912
:107110008005F3D561688803800F032805D13268A4
:107120000005824301400A433260286903226168F6
:107130001204114008432861002F04D0B16B0120D4
:1071400000078143B1632078C00705D0E868A168D3
:10715000800880000843E8602078800705D5E8684B
:107160000C218843E1680843E8602078400706D591
:10717000E86803218902884321690843E860207890
:10718000000706D5E86803210903884361690843BD
:10719000E8602078000606D5E86803218904884362
:1071A000A1690843E8600020F8BD000040100240DB
:1071B0000070004088130000F8B50E46050038D076
:1071C0005E480068C007C00FB04214D25B4C206814
:1071D0004008400030432060FFF752FC074605E0BE
:1071E000FFF74EFCC11B564881427AD82068C00781
:1071F000C00FB042F4D12878524C800705D5E06822
:10720000F0218843A9680843E0602878C00752D07D
:107210006868022806D0032807D0216801280AD010
:10722000890504E02168890301E0216889010029BA
:1072300003DB0120F8BD4907F9E7E1688908890007
:107240000143E160FFF71CFC0746686802280AD08A
:10725000032814D001281ED029E0FFF711FCC11B20
:10726000374881423DD8E0680007800F0228F4D1FA
:1072700021E0FFF705FCC11B3148814231D8E068AD
:107280000007800F0328F4D115E0FFF7F9FBC11BBD
:107290002B48814225D8E0680007800F0128F4D1EF
:1072A00009E0FFF7EDFBC11B2548814219D8E068D2
:1072B0000007800FF5D121480168C907C90FB14205
:1072C00017D901684908490031430160FFF7D8FB2D
:1072D000074608E005E0FFF7D3FBC11B18488142D1
:1072E00001D90320F8BD15480068C007C00FB0429F
:1072F000F1D12878400706D5E068072109028843C4
:10730000E9680843E0602878000707D5E0680721AE
:10731000C90288432969C9000843E06000F03AF8CF
:10732000E168094A0906090F515CC840074908602D
:1073300007480068FFF7C6FBF8BD000000200240C8
:1073400088130000001002403AB0000870010020CD
:1073500068010020044805490068C968044A4905D5
:10736000490F515CC8407047700100200010024076
:1073700053B00008044805490068C968044A8904F4
:10738000490F515CC8407047700100200010024056
:1073900053B0000870B51A4AD3681A490C20184037
:1073A0008D0004280CD04E00082810D00C2810D0D6
:1073B00050680004410F0120C003491C884070BD83
:1073C0001068C00601D5084670BD284670BD30461D
:1073D00070BD98020C4C000F205C1B029C0FD36800
:1073E000641CDB0301D5314603E01268D20600D4E9
:1073F000294602F084FE22460023FDF78FFE70BD71
:107400000010024000093D004AB00008FEB505002A
:107410007ED0FE4CE7680C20E6680740012000049F
:1074200006402878C00747D0082F05D00C2F0AD176
:1074300001200004864206D1206880033CD568689C
:107440000028E5D038E0012069680004814203D1BA
:1074500021680143216011E0052301221B049204ED
:107460009942216802D111432160F1E781432160F3
:1074700021680140009120689043206068680028DE
:107480000DD0FFF7FDFA009005E0FFF7F9FA00993B
:10749000401A64287BD820688003F6D50CE0FFF7FB
:1074A000EFFA009005E0FFF7EBFA0099401A642824
:1074B000F0D820688003F6D42878800756D50923B1
:1074C000E868042F0DD00C2F01D1002E09D0002820
:1074D0003CD02168994301432160FFF7D1FA064669
:1074E00028E02168490701D5002891D061681F2252
:1074F000120291432A691202114361602168994383
:1075000001432160FFF746FFE16809060A0F00E02A
:107510008BE1BF49895CC840BE490860BE4800682D
:10752000FFF7D0FA002873D120E0FFF7A9FA801BFB
:107530000228AFD820684007F7D560681F210902EC
:10754000884329690902084360600FE02068400809
:1075500040002060FFF794FA064604E0FFF790FA37
:10756000801B022896D820684007F7D42878C006E8
:1075700060D5002F0CD0A86900284AD02068FF21D0
:10758000013108432060FFF77BFA06462EE0C1E098
:107590002068800502D5A8690028A6D06068072168
:1075A00049038843296A084360606068297F0002B4
:1075B000000A090608436060286A410B0120C003E5
:1075C000491C8840E16809060A0F9149895CC84056
:1075D0009049086090480068FFF774FA002817D1B6
:1075E00028E0FFF74DFA801B0228A2D8206880050A
:1075F000F7D56068072149038843296A084360601A
:107600006068297F0002000A09060843606011E0F3
:10761000E2E02168FF20013081432160FFF730FA6A
:10762000064604E0FFF72CFA801B022872D8206877
:107630008005F7D42878794E000724D5686900289A
:10764000306910D0012108433061FFF719FA00902A
:1076500005E0FFF715FA0099401A02285AD8306958
:107660008007F6D50FE0400840003061FFF708FAC8
:10767000009005E0FFF704FA0099401A022849D863
:1076800030698007F6D42878400766D5002002903C
:10769000A06BC00006D4A06B012109070843A063BA
:1076A000012002905E480168C90511D40168821565
:1076B00011430160FFF7E4F9009005E0FFF7E0F9FE
:1076C0000099401A642825D855480068C005F5D5AA
:1076D000FF20AA680130824203D131690143316140
:1076E00011E001218902002A07D005231B029A42DA
:1076F00003D132690A433261EFE732698243326172
:10770000306988433061A868002810D0FFF7B8F9C5
:10771000009008E05FE0FFF7B3F901460098091A0E
:107720004048814257D830698005F4D50DE0FFF715
:10773000A7F9009006E0FFF7A3F90099411A39482C
:10774000814248D830698005F5D40298002804D0D9
:10775000A06B012109078843A063686A002866D0EE
:107760000C2F3ED0012636060228206805D0B043F3
:107770002060FFF785F905462FE0B0432060FFF752
:107780007FF9074604E0FFF77BF9C01B022822D8E7
:1077900020688001F7D4E96AA86AE2680843296B87
:1077A000FD231B049A4311430843E06020683043E3
:1077B0002060FFF765F9054604E0FFF761F9401B1B
:1077C000022808D820688001F7D530E0FFF758F983
:1077D000401B022801D90320FEBD20688001F5D49A
:1077E00025E00128F8D0E06801210904AA6A0140D7
:1077F00091421AD10F218904EA6A0140914214D1C1
:10780000032189050840296B88420DE000100240E1
:107810003AB00008700100206801002040100240CA
:10782000007000408813000001D00120FEBD002040
:10783000FEBDF8B504000ED0FF27606A05370025AD
:1078400000280AD02561656126464036A562707C15
:10785000002807D00AE00120F8BD6068B842F3D0E4
:10786000E561F1E73574204600F03EF802217174BD
:107870002068026840239A4302602123A26860685E
:107880009B021A4038401043E3688A0213401843B1
:1078900023690B40217D1843C907C90F0843A1691B
:1078A000931019400843E169382319400843216ABD
:1078B000802319400843A16A9300194008432168B6
:1078C0000860A0690421000C0840616A1023194077
:1078D0000843216848602068C1699143C1616565BA
:1078E000012070740020F8BD10B586B00446142144
:1078F0006846FDF75CFC10492068884219D10F48A2
:10790000416B821411434163C16A01221143C16278
:10791000C06A002110400590E020009002200190F4
:107920000320039002910491052069460007FEF7A9
:10793000D7FF06B010BD000000300140001002402B
:10794000094910B5401E884201D9012010BD074CDD
:1079500060610321081F02F0F7FB0020A0610720EF
:107960002061002010BD0000FFFFFF0000E000E0EC
:107970007047704770470000F8B502680446D06948
:1079800011689668814B05461D402023002D6CD060
:10799000F7077F4DFF0FBC460D402F4379D025469A
:1079A000C7078035002F06D0CF0504D50127176201
:1079B0002A683A432A60820708D5F20706D027686A
:1079C00002223A622A6804273A432A60420708D50D
:1079D000F20706D02668042232622A680226324361
:1079E0002A6002070AD50A461A406646324305D085
:1079F0002668082232622E6816432E60020508D5DA
:107A00004A0106D501222668D20232622A681A4348
:107A10002A602A68002A30D0800606D5880604D558
:107A2000616E002901D0204688472868216889684E
:107A3000490602D42821084225D0204602F0ABF89E
:107A400020688168490619D5826840218A4382608E
:107A5000206F002812D04F498163206FFEF7A6FDEA
:107A600000280AD0206F816B06E0850611D58D06AF
:107A70000FD5616E77E020468847F8BD2046FFF7B6
:107A800079FFF8BD05E02046FFF774FF002028606D
:107A9000F7E7256E012D56D1C50654D5CD0652D532
:107AA000102616622068816825464906403500295F
:107AB0002ADA226F116849680904090CE1D02F8B7A
:107AC0008F42DED9698311680968890617D4016875
:107AD0003201914301602068816849084900816052
:107AE00020688168402291438160E367002020661E
:107AF00020680168B1430160206FFEF735FD288BD7
:107B0000698B401A81B21AE0298B6A8B891A6A8BB9
:107B100089B2002AB5D00029B3D00268FF252135EB
:107B2000AA43026020688268520852008260E367BC
:107B300000202066606620680268B243026020462A
:107B4000FFF716FF9DE7C50208D5750206D501208F
:107B5000000510622046FFF70CFF92E7050605D5E9
:107B60000D0603D5A16E002985D18AE7400688D588
:107B7000480686D5116820464024A14311608367DA
:107B80000021816600F043F97BE700000F08000048
:107B900020010004BD9A000810B5040003D0A06FB6
:107BA000002802D007E0012010BD002174200155FB
:107BB000204600F027F82420A067206801684908C3
:107BC00049000160204602F039F80128ECD0606AD3
:107BD000002802D0204601F05BFE2068416809229F
:107BE000D20291434160206881682A2291438160DA
:107BF00020680168012211430160204601F0AEFEB9
:107C000010BD0000F0B587B0064614216846FDF7A8
:107C1000CEFA2C493068884251D12B48416B012261
:107C2000920311434163C16A01221143C162C06AD8
:107C300000251040059003204002009002200327F9
:107C400001A9A1C104200490052069460007FEF7A0
:107C500047FE1F4C1D48A560E56081C48027E56094
:107C6000A7602020256160610002A0611848083CDF
:107C7000FEF716FD002801D0FEF700F83467A66273
:107C8000144C1248214614382060032060601020F4
:107C90000831A1C16561A561E56120462562FEF755
:107CA000FFFC002801D0FDF7E9FFF4660022012166
:107CB0001B20A662FFF770F91B20FFF761F907B0E0
:107CC000F0BD0000003801400010024030000240CA
:107CD0000C1700205417002070B5C36F202B27D13C
:107CE00000290BD0002A09D0012483682403A34271
:107CF00006D10369002B03D1CB0701D0012070BD51
:107D0000034660331C7D012C12D001241C75002316
:107D10000366084C0368A34207D05C68240204D5BC
:107D20001C680125AD062C431C6002F087F870BD6D
:107D3000022070BD0048004070477047FFB5044600
:107D4000806F83B017460D4620285ED1002D0AD0E3
:107D5000002F08D0A168C001814207D12069002806
:107D600004D1E80702D0012007B0F0BD2046603002
:107D70000090007D012848D0009801210175002065
:107D8000802108512120A067FEF77AFE2646403662
:107D90000190378277820120A1680003814202D1DD
:107DA0002069002805D02F4600250099002008757D
:107DB00011E00027F9E700228021204602F084F834
:107DC000002815D1002F15D02168387888627F1CD3
:107DD000708A401E7082708A019B0028069800906D
:107DE000E9D100224021204602F06EF8002808D098
:107DF0000320B9E728882168C005C00D8862AD1C42
:107E0000E6E72020A0670020AEE70220ACE770473D
:107E1000034D044C04A002F051F9E560FAE70000BC
:107E20000400FA0500ED00E0486172644661756C7B
:107E3000745F48616E646C65722E0D0A000000006C
:107E400070B586B014216846FDF7B1F901240B48DE
:107E50000526C4800A48E50244833607224629469F
:107E60003046FEF706FE0021029103910095019431
:107E700069463046FEF734FD06B070BDE40D0020C3
:107E80002401002070B501240E4DA40300222146D8
:107E90002846FEF7EEFD002204212846FEF7E9FD04
:107EA0000A2002F0D2FA012221462846FEF7E1FD1F
:107EB0000A2002F0CAFA002221462846FEF7D9FD20
:107EC00070BD00000004005070B501240E4DA403E5
:107ED000002221462846FEF7CCFD01220421284637
:107EE000FEF7C7FD0A2002F0B0FA0122214628461B
:107EF000FEF7BFFD0A2002F0A8FA0022214628461C
:107F0000FEF7B7FD70BD000000040050F1B500247D
:107F10000126154F2546B603002231463846FEF7A6
:107F2000A8FD0A2002F091FA012231463846FEF7F8
:107F3000A0FD6006040E04213846FEF78DFD0028E2
:107F400001D0641CE4B2052002F07FFA6D1CEDB292
:107F5000082DE1D30098002803D0FFF793FF2046B7
:107F6000F8BDFFF7B1FFFAE700040050F8B50126AD
:107F7000154F0546B603002231463846FEF779FD17
:107F80000024E80901D0012200E000220421384643
:107F9000FEF76FFD6806050E0A2002F056FA012270
:107FA00031463846FEF765FD0A2002F04EFA0022FF
:107FB00031463846FEF75DFD0A2002F046FA641CA1
:107FC000E4B2082CDDD3F8BD0004005070B50D4CB0
:107FD000012204212046FEF74CFD0122950329468B
:107FE0002046FEF746FD002204212046FEF741FD13
:107FF0000A2002F02AFA002229462046FEF739FD1F
:1080000070BD00000004005070B501240E4DA403A3
:10801000002221462846FEF72CFD00220421284696
:10802000FEF727FD0A2002F010FA01222146284619
:10803000FEF71FFD012204212846FEF71AFD0A2043
:1080400002F003FA70BD00000004005070B5144D3A
:108050000024012204212846FEF70BFD062002F031
:10806000F4F90122960331462846FEF702FD062068
:1080700002F0EBF907E0641CE4B2FA2C03D9FFF735
:10808000C3FF012070BD04212846FEF7E5FC00284F
:10809000F1D1002231462846FEF7EBFC002070BDEE
:1080A00000040050F8B501F08BFC01F0BBFC3B482C
:1080B0000068C069FDF7A4FF394D3A4E2870402191
:1080C0003046FEF7C9FC77010024002827D0364847
:1080D0000460A879002803D10120A87101F056FF9F
:1080E00080213046FEF7B8FC002806D00022082187
:1080F0003046FEF7BEFC012205E001220821304691
:10810000FEF7B7FC0022052039460007FEF7B1FC58
:10811000264D274EA88C274F012803D01CE0AC71B8
:108120000022EBE724486946088072B68021234884
:10813000FDF7BCFD002804D0022269461F48FDF768
:1081400059FE62B61EA001F0B9FFAC8402F0F6FE43
:10815000642002F073F9FE60688C012809D113488D
:108160006C844038048002F0E9FE642002F066F975
:10817000FE60288C012806D12C8402F0DFFE6420EA
:1081800002F05CF9FE600948114A403801889142CA
:1081900002D1C088002800D1FE60F8BD88160020FA
:1081A000240100200004005060010020E40D0020A4
:1081B0000400FA0500ED00E0AAAA0000384A000811
:1081C000BDF8C8EBC9FDBCB6C4A3CABD0D0A00000A
:1081D000AA55000038B500246946202000F0AAF80E
:1081E00068460078572800D001246946212000F015
:1081F000A1F868460078032800D0012469462220AF
:1082000000F098F868460078402800D001246946BC
:10821000232000F08FF868460078082800D0012459
:108220006946302000F086F868460078AA2800D019
:1082300001246946322000F07DF80C486946008F21
:108240000978884200D001246946332000F072F892
:1082500006486946403040880978884201D1002CA0
:1082600002D004490248C86038BD0000A40D0020B7
:108270000400FA0500ED00E038B55721202000F099
:108280007AF80321212000F076F84021222000F026
:1082900072F80821232000F06EF8AA21302000F0A7
:1082A0006AF81048018F142901D8002901D1012151
:1082B00001870C4C40346188142901D8002901D170
:1082C00002216180008FC1B2322000F054F8A17801
:1082D000332000F050F8684600F006F80A2002F05B
:1082E000B4F838BDA40D002010B501460F2000F0F1
:1082F00021F8002800D0012010BD10B50446FFF77A
:1083000065FE3220FFF732FEFFF7A0FEE0B2FFF776
:108310002DFEFFF79BFEFFF759FE3320FFF726FEE9
:10832000FFF794FE0020FFF7F1FD0446FFF76CFE17
:10833000204610BD10B50C46FFF7DFFF207001206E
:1083400010BD70B50D460446FFF740FE3220FFF722
:108350000DFEFFF77BFEE0B2FFF708FEFFF776FEAB
:108360002846FFF703FEFFF771FEFFF74DFE0A20D8
:1083700002F06BF870BD10B5FFF7E3FF012010BDF0
:1083800010B50248FEF7BBFC10BD0000C015002070
:10839000FEB50446002772B6334A01688B1804D133
:1083A0003248C76803208004074088680190C86885
:1083B000009048698E69002B08D12C4940398B6A9E
:1083C000CD042B438B628B6AAB438B6201463143F6
:1083D0003CD025492368CB4205D12449CA680323F0
:1083E0009B049A43CA6025462035002810D0216896
:1083F0000A6901231A430A6121684861082120465D
:1084000000F036F8032800D1A873216808204860DE
:10841000002E10D0206801690122114301612068FB
:1084200086611021204600F023F8032800D1A873AC
:108430002168102048600C482168C14206D10B48D1
:10844000C1680322920491433943C16020680169E5
:1084500049084900016121680198886021680098F5
:10846000C86062B6FEBD00000084FFBF401002403D
:1084700070B506460B480D46002409490068FCF714
:1084800037FE7D21C90048433168401E00D10324D6
:108490000B682A469A4301D00028F6D1204670BDC9
:1084A000204E0000700100201CB5002116480091EC
:1084B000144A01910260C163120542608160072283
:1084C0008263012202610246C16020321170FF23E3
:1084D0005170C2334362816211730163816104226E
:1084E00041634261C161FDF7A5FE08480090801319
:1084F000019069460448FDF74DFE00210248FDF752
:10850000F3FD1CBD0024014064150020020000049E
:1085100008B50848016B012211430163006B01217A
:108520001040009000220A20FEF736FD0A20FEF7D8
:1085300027FD08BD00100240F0B587B01421684641
:10854000FCF735FE4648C26A04210A43C262C26A89
:108550000A400592C16A80263143C162C16A314036
:108560000591C16A01242143C162C16A214005917C
:10857000C16A02252943C162C06A2246284005908B
:10858000052010210007FEF774FA0122354936480C
:10859000FEF76FFA002235493348FEF76AFA912157
:1085A0000520002209020007FEF763FA3048019017
:1085B000002705206946029700940007FEF790F90E
:1085C0002C480090112001900320039002976946E7
:1085D0002548FEF785F910206A46039591C20520CB
:1085E00069460007FEF77CF9112001900297694661
:1085F000039700941C48FEF773F91F4801906946E1
:10860000009502941848FEF76BF9402000906946E7
:10861000019702951448FEF763F91848694691C11D
:10862000694611480397FEF75BF9912000026946FD
:1086300091C10520694600070397FEF751F9694685
:108640000948019700960294FEF74AF90022012199
:108650000520FEF7A1FC0520FEF792FC07B0F0BD57
:1086600000100240054200000004005008300000E5
:10867000000011100440000000002110083200002A
:1086800010B50F4C0D482060FF20053060600020C1
:10869000A060E06020616061E06101212062490228
:1086A0006062A161A0620720E0622046FFF7C1F886
:1086B0002068016840221143016010BD0030014074
:1086C000F015002000B585B014216846FCF76FFD59
:1086D0000E480D490160E12149024160002181609D
:1086E000C160016181610C22C1614261016230217E
:1086F00041620121090381634900C163FFF74CFA1C
:1087000001F03EFC05B000BD003801408816002095
:1087100070470000F0B589B00A2002F07FF97D2093
:10872000400102F095F9FF4C0025A570FE48206637
:10873000607C0C2801D30B20607460790A2801D971
:108740000A206071F948E570F94E00783071F949F6
:10875000A079097840000843A17D89000843F071A1
:10876000E06BF070010A3172401CE0636079B07414
:1087700042003046F0491330FCF700FD6079EE49C5
:1087800082004000801960311330121DFCF7F6FCA6
:1087900060790621420048438019E8491730921C4D
:1087A000FCF7ECFC2E20205E002803D0E449098A67
:1087B0000818E0856079DB49C000223182190B7B03
:1087C00053764B7B937606227272DE4A1D30127806
:1087D000B272A28C3273D64A0B79133A1375497967
:1087E00051750022D24902F003FA60790021C000DD
:1087F0001D3002F00FFAD448FEF75CFB01272085FC
:10880000BF0309E0D048FEF755FB80B22085E18E1A
:10881000FF392D39884206DB81B2E08E8142F1D3E7
:10882000C0198142EED8022002F048F9C048012662
:10883000C571A574A5732674E573C348FEF73AFBAA
:1088400060850746E5706079FCF724FFBF4AC04B9E
:10885000FCF71AFE01F08EFD0022BE4BFCF762FD14
:10886000FCF75EFF0006C00CC01980B2F103A085C2
:10887000884201D3401AA085B748E0642079401CA3
:108880002071B148FEF716FB2085AB48A54F643830
:1088900040370690B1E1AC48FEF70CFB20850BE0B9
:1088A000A948FEF707FB80B22085A18D884203D33B
:1088B000AA4A8918884207D300210F2002F02EF817
:1088C000A74920640842EBD0206C411C1FD0400413
:1088D0007ED58122D20100210F2002F05EF9002115
:1088E000102002F01BF841069348490E00227C3804
:1088F000E16502F049F8002002F0AAF8002002F039
:108900005CF88D487C38417A0729C3D101E001F039
:108910003DFC02229349401DFCF754FC0028B9D1CC
:1089200002F0C9F9E167A06702F0B2F97D4B80332C
:1089300003C3E0788049401CE07083390B7A6846B5
:108940000370497A417000880390E18C88427DD1A0
:10895000774985488C31C98E0180754871498C30C2
:10896000008F48847848FEF7A5FA208501F0E8FEDC
:108970006C48FF2280300168406852040023891847
:1089800058410206080A10434108490000900A0EA7
:10899000080264498031CA6088606548E36F0A3024
:1089A000A26F02F05DF960798100614808185D49A5
:1089B000163080310CC902F053F95A488030C36830
:1089C00082685B48123002F04BF90821584800E0F9
:1089D00006E14172B430C07C0009607514D056487D
:1089E000022260497738FCF7EDFB00280CD1504893
:1089F000A674C671E06D50491638C2B26639C81DFA
:108A0000E274FB30FCF7BAFB607900228000484931
:108A10001C3002F0EDF86079002180001C3002F07B
:108A2000F9F8009801F0F3FF012002F047F82073F5
:108A300002214E48FEF710F800281DD000213D48C5
:108A400001703B498C31488E049000E05AE0388137
:108A5000888E78818446A06CFF310531E06408601F
:108A6000DC392065C97C0907090F032900D021756D
:108A7000E16D1C2902D015E00121E0E72C49294ACB
:108A80008C31C98F1186069B2C4A1B881380884223
:108A900007DD002805DD002903D0207E401C20765C
:108AA00000E025762571A6730498B8816046F881A8
:108AB000E673608C2E49FF30C33080B260848842F8
:108AC0000CD949424018608427487D220188D20091
:108AD000491C89B20180914200D3058022487D2142
:108AE0000088C9004843618C4018606500F076FD3D
:108AF000207B002805D100210F2001F00FFF000688
:108B0000F9D583E0FDF792F90B4A03219032115415
:108B100007498C314A8E3A81898E7981E26D1C2A0F
:108B20002ED127E0580000203F420F0024010020F2
:108B3000181200205C01002048130020841400203B
:108B4000E40D002034010020C0150020B81E85EB84
:108B500051B8CE3F00000840A0860100983A0000BE
:108B600000D027244C0100205801002000040050B0
:108B7000E7030000624B4200D318069A12885A801D
:108B80008000604B5F4AD43B02905E4982189B8F05
:108B9000138030314118A26C4A605B4940185B4930
:108BA00016300CC902F05CF8216EA06C884207DA1E
:108BB000544A02995158012902D12066039905911E
:108BC0005049029A8958814217DD012915DD214655
:108BD000002812DD0398C8840220087065730CE039
:108BE0004B4A00210F2001F0D8FF6079E178401C4A
:108BF000814202D0002001F0E0FE208DA18D88424C
:108C000000D248E6434A89188842FAD8A07B012856
:108C100001D00220A07301F093FD3D4A00210F20F6
:108C200001F0BBFF2179002917D03B480288900052
:108C300013188B4200D22570002000F0E9F8A07CC8
:108C400000283BD02F496C310B78A37248786072B2
:108C50008A782272022B17D030E0E16C226E323912
:108C600020468A420EDAC1792B4A491CC9B2C17129
:108C7000128852008A42E2D20599C1840221017011
:108C80006573DCE7E571DAE710280ED0C82815D245
:108C9000224BC91C1D60224B1818FCF76FFA02F01A
:108CA0004DF9642001F0CAFB31E61E4D28684000F2
:108CB000000E03D1C878FCF7D2FC2860002023788E
:108CC000627B657910E00F4E0E4F4100303E183F39
:108CD000765A7F5ABE4205D00A4F0223002201264F
:108CE000483F7E52401CC0B2A842ECD3237062734E
:108CF000074A002180320F2001F04FFF09B0F0BD7C
:108D0000841400207813002018120020D8000020BE
:108D100000D02724983A0000340100206001002090
:108D2000A40D002050010020F8B52E4C0546E06E41
:108D30002D4A281A411E2067914215D21A21615EE0
:108D4000081AFCF793FC294A294BFCF79DFB0646C1
:108D500032200F46205EFCF789FC32463B46FCF78A
:108D6000E1FAFCF7B9FC6086002060761D481C2300
:108D7000C35E828C1F48008884461F4806881DE019
:108D80006046484380181D4F80B2388030277843B2
:108D90006427643078431A4F6066C01985420BD24D
:108DA000C8B2184932220880606EA25E411BC91801
:108DB0008918A166E066F8BD491C6176617EB14202
:108DC000DED33020424310486421101848430F4935
:108DD0004118E16660663221401B615EC018401890
:108DE000A066F8BD58000020CF0700009A99999915
:108DF0009999B93F46010020340100205A01002012
:108E000078ECFFFF4401002074270000C0BDF0FF94
:108E1000FEB5294D2988491C8FB228492F800E881C
:108E2000FCF724FC264A274BFCF72EFB019100900F
:108E300025483146FCF75CF9244C218F4218B74293
:108E400006D3002028802248019E1018009D02E0D1
:108E50001046019E009DFCF71DFC33462A46FCF798
:108E600061FAFCF75DFCA086012580B2ED03A84203
:108E700001D3401BA086E08BFCF70CFC154A164B77
:108E8000FCF76AFB0646A08E0F460090FCF702FC3A
:108E900032463B46FCF746FAFCF742FC80B2E086DD
:108EA000A84201D3401BE0860C490098096848613C
:108EB00000982087FEBD00004401002034010020FE
:108EC0001904560E2D624040E17A0000580000203F
:108ED0001F050000F853E3A59B843E40C015002009
:108EE00070470000F0B589B0002004900A2001F01E
:108EF00095FD7D20400101F0ABFDB348002282705A
:108F0000C16BB34C491CC163B049C38D098A254666
:108F1000C918C1852146C2751331079147310391A4
:108F20006D393135AB4F223005910290A64E0F219D
:108F3000A948717100782071A84AB0791278400070
:108F40001043B27D92001043E071B08FE070000AD0
:108F50002072A17431461E229C310798FCF70EF94D
:108F6000402228469E49FCF709F9029903980A7B9A
:108F7000C274497B0175092060729A480078A0721A
:108F8000B08C2073F07D410030469C300918059864
:108F90000A78027549784175762000228C4901F0E3
:108FA00027FE70790621484300211C3001F032FE73
:108FB000022001F083FD00210F2001F0AFFC3842B8
:108FC0003064F8D0306C411C18D040047ED581222A
:108FD000D20100210F2001F0E0FD0021102001F05E
:108FE0009DFC41067A48490E0022B43001F0CCFCC9
:108FF0007748B430417A022902D0BDE001F0C6F8CA
:1090000002227949401DFCF7DDF80028F5D16E48B1
:109010000222C07D41006C489C3009186C48B53074
:10902000FCF7D0F80028E8D101F045FE664AD16788
:10903000906701F02DFE644A803203C20498002834
:109040002CD1012004906248684E8C30C08E60495B
:1090500030805D488C31098F41846548FDF72AFFD7
:109060005949644A0885488CFF30C33080B248842F
:1090700090420CD952428018488430885D4A401C86
:1090800080B20B323080904201D300203080308893
:109090007D22D20050434A8C801848654C4869466E
:1090A0008C30428E0A80808E488049490422B53136
:1090B000C81FFF38FCF762F84348494AC07D009951
:1090C000800011504049803103C900E075E0FF2362
:1090D0005B040022C01851410906060A0E433046BF
:1090E00001F095FC710849000A0E08023649002675
:1090F0008031CA6088603448C36F826F3448483812
:1091000001F0AEFD304880300CC83148443801F0E1
:10911000A7FD2D488030C36882682D48403801F093
:109120009FFD2B49002252393C2001F061FD0021B6
:109130003C2001F06FFD012001F0C0FC22490873C2
:1091400008468078401C887001210520C90300076B
:10915000FCF780FE1C48007B002805D100210F2071
:1091600001F0DCFB0006F9D5802200210F2001F080
:1091700014FD1548467002E013490120487012485A
:10918000C17D491CC9B2C1750F2900D2CEE6049831
:10919000002810D10C4A1849908C002802D00B8866
:1091A000984201D908889084144980B20988401EE9
:1091B00048431349088009B0F0BD124A00210F202E
:1091C00001F0EBFCD8E7000058000020E40D00207F
:1091D0001812002000D02724240100205C01002068
:1091E00034140020340100204C01002058010020DC
:1091F000C0150020E7030000300100202E010020F0
:109200002C01002000902724F8B53249304808602E
:1092100001F036FE304800F0A1F9304CE0822E48D3
:10922000801C00F09BF920832B48001D00F096F96C
:10923000608323212A480901418001464031097990
:10924000284F0906090E617006D1C7800121C18728
:109250000A21418700218187234AC18E1170C18F65
:109260002171818F6171817AA17085880521A56244
:109270006181C6883046FBF73BFFA0810146284646
:10928000FBF736FF8800081885B216482581684329
:10929000FCF700FA154A164BFCF75EF9FCF740FAAA
:1092A000E081658231463846FBF722FF2082014685
:1092B000C820FBF71DFF608401202084FCF7CEFD51
:1092C000A082E2890B490C48FDF7F8FDF8BD0000CB
:1092D000AD9F000850000020004F0008240100202E
:1092E000A40D0020E803000000000020F853E3A5CF
:1092F0009B843E40FF7F0000C0150020F8B5744CF1
:1093000000202071734D01202880734EC8203080CA
:10931000E07A401CE072C00706D0A08C411EA184F8
:10932000022801D2C820A0840120C043FFF770FDAD
:109330000A2001F073FB7D20400101F089FB02212E
:109340006648FDF789FB00287ED000206449800034
:109350000978654F49000843624909780843B872A3
:10936000102078726148C1887D20C000FBF7C0FEE4
:1093700078735F485D490078B87338460B308A7857
:109380000270C97841705949421C20310B7ED3705C
:10939000497E11715549D01C22310B7E5371497E93
:1093A0009171524940310A7C0271497C417100221D
:1093B0003946172001F01CFC0021172001F02AFC7F
:1093C000022001F07BFB4B4F00210F2001F0A6FA99
:1093D00038422064F8D0206C411C77D0400471D50D
:1093E0008122D20100210F2001F0D7FB00211020A3
:1093F00001F094FA41063C48490E0022B430E16580
:1094000001F0C2FA384FB437787A11285AD10222C3
:109410003949781DFBF7D6FE002853D1F81F027A90
:1094200069460A70407A4870B97A2980C820FBF7EB
:109430005FFE3080387BA0843846304D2838C08E9F
:1094400028802348394600E03EE02839098F4184CE
:109450002B48FDF72FFD2085608C2A49FF30C33053
:1094600080B2608488420CD94942401860842888C0
:109470002449401C80B20B312880884201D300204F
:10948000288028887D21C9004843618C4018606588
:1094900000F0A4F868460088E0841349B87CC7311E
:1094A0006071420008460D466930FBF767FE60793F
:1094B000294642001448FBF761FEA08CFF2801D02A
:1094C00003202070F8BD01E001203FE700F05EFEC0
:1094D0005800002034010020460100200004005004
:1094E000280100202901002018120020A40D0020CE
:1094F0000000002000D027244C010020580100204B
:10950000C0150020E70300006013002070B586B08E
:1095100014216846FBF74BFE01250F4EED03002298
:1095200029463046FDF7A5FA012000240190029457
:109530006946009503943046FDF7D2F90320019067
:1095400002946946009503943046FDF7C9F902205C
:1095500000F074FF06B070BD000400500088704732
:1095600070470000F8B5044600206A461080194D87
:1095700055222A70AA226A700322AA70661DEE7014
:109580002A716971144A49008918AC712246E81D94
:10959000FBF7F4FD002007E029186A468978128855
:1095A00089186A461180401CB042F5DB611DA81C79
:1095B000FCF7B2FA01466846018029190078C871A3
:1095C00068464078087221460931024800F004FBE1
:1095D000F8BD0000FE140020A40D0020FEB5FFF72A
:1095E000A3FB2548FDF766FC244C86B226856079EE
:1095F0000A21081AC000FCF739F807460191A06E4D
:10960000FCF748F81E4A1F4BFBF7A6FF00900D46DB
:109610003046FCF73FF82B46009AFBF783FE3A46AC
:10962000019BFBF77FFEFCF77BF885B2A586E08BFC
:10963000FCF730F8124A134BFBF78EFF06460F4635
:109640002846FCF727F832463B46FBF76BFEFCF753
:1096500067F881B20120C003E186814201D3091A73
:10966000E186854201D3281AA0860349A08E0968A5
:1096700048612087FEBD0000C01500205800002072
:10968000F853E3A59B843E40034A1168382389B20E
:1096900099430143116070470030014010B5FDF758
:1096A000F5F910BD10B59AB034216846FBF77FFD7F
:1096B00014210DA8FBF77BFD1C2112A8FBF777FDF9
:1096C0001B4801680324E402A143C2148918016005
:1096D000FDF76EFC17480169A14301610620009067
:1096E000FF200130029001200390102004900220FE
:1096F000099040040B90000100240C900A946846E5
:10970000FDF784FE0F200D9003200E900F9410940F
:10971000012111940DA8FDF74FFD81201290032027
:1097200080041890149412A8FDF794FC1AB010BD90
:10973000007000404010024010480168821511433B
:109740000160C1680E4A1140C16001680D4A1140B4
:109750000160816849084900816001680122920422
:1097600091430160C168FD2212049143C160002150
:1097700001610649044888607047000000100240FB
:109780000C40FF88F6FFF6FE0050000800ED00E0F8
:10979000F8B5102405252D07AC62AF20800000F03D
:1097A00054FEAC6101F0CEF82F4C304F304E606764
:1097B0000EE001F0C7F86067FEF774FC606C411CB6
:1097C0006164142804D92BA000F078FC2D48C760F0
:1097D000606FB042EDD10026666420780127FF0358
:1097E000030000F0A4FC05040C192D303200012206
:1097F00039462846FDF73DF9FFF780FD06E00122D6
:1098000039462846FDF735F9FFF76CFB002239464B
:109810002846FDF72EF918E0607B0122401C60739A
:1098200039462846FDF725F9FCF734FB0022394676
:109830002846FDF71EF9607B052806D9267004E04E
:10984000FEF768FF01E0FFF74DFB02210E48FDF730
:1098500003F9002805D000200C49087000F058FFDB
:10986000F8BD0120F8E70000580000200400FA05C8
:109870003001CADE4457204944204552524F522EEF
:109880000D0A000000ED00E0000400505C01002023
:1098900010B5818CC90707D001684A6801235B04B1
:1098A0009A43836A1A434A60818C890707D5016805
:1098B0004A6801231B049A43C36A1A434A60818C95
:1098C000490707D501684A6801239B049A43036B43
:1098D0001A434A60818C090707D501684A68012349
:1098E000DB039A43436B1A434A60818CC90607D550
:1098F0000268916801231B039943836B19439160AC
:10990000818C890607D501688A6801235B039A4325
:10991000C36B1A438A60818C490612D503685A6862
:1099200001210905046C8A4322435A60026C8A4271
:1099300007D10268516803235B059943436C1943BF
:109940005160818C090607D501684A680123DB0450
:10995000806C9A4302434A6010BD0000F8B504468B
:10996000002680300660FDF78BF805462068006809
:10997000124F000709D501212B4600224905204638
:10998000009700F0A1FA00280DD120680068400778
:109990000BD501212B46002289052046009700F0B7
:1099A00093FA002801D00320F8BD2020A067E067CB
:1099B0002666603426750020F8BD0000FFFFFF0119
:1099C000F8B5154CC826E078002823D16079002826
:1099D00020D101206071114D686B0027002818D03C
:1099E000686BC821081A0FE00D48E168405C6169A6
:1099F0008847E068401CE060E068C82800DBE7605A
:109A0000696BC820401A761EE168814201D0002EA1
:109A1000EADC6771F8BD00003C0000200000024055
:109A2000DC0C002070B5224CE07800283FD1207972
:109A300000283CD1012020711E4EF1690025090645
:109A4000002933DA2156625791420AD1F069400663
:109A50002CD5A079002829D0A5712089401C20810F
:109A600024E0A179002903D1A0710A2000F0EDFCC7
:109A700000202056CC2148430F4942182069121873
:109A80001279B262401C00222061A256CC235A43B4
:109A9000895881420ADC25612078401C207020789A
:109AA0000E2800D12570A078401CA070257170BDD3
:109AB0003C00002000380140B401002010B5806A4D
:109AC0000022014640314A834A82FDF753FF10BD10
:109AD00070B5846AA06FE56F216889680026090661
:109AE000002906DA212804D152200653204600F02E
:109AF0006BF820688068400606D5222D04D15A20D4
:109B00000653204600F047F82046803001681022B6
:109B1000114301602046FDF72DFF70BD10B50146D1
:109B20000968806A096889061CD400225A210A52F1
:109B300001680A68FF2301339A430A6001688A6852
:109B4000520852008A6001688A6840239A438A60FA
:109B50002021C167016E012904D101680A68102320
:109B60009A430A60016E012902D0FEF7E5F810BDA4
:109B70005821095AFDF7FCFE10BD10B5806A016E30
:109B8000012902D0FEF7D9F810BD5821095A490819
:109B9000FDF7EEFE10BD01680A68FF2321339A43EA
:109BA0000A6001688A68520852008A60016E0129C1
:109BB00004D101680A6810239A430A602021C16712
:109BC000002101664166704701680A68C0239A4314
:109BD0000A6020218167704770B5164CE278002A30
:109BE0000CD12279002A09D10122E2700025C8296E
:109BF00003DC0222A256002A01DCE57070BD0123BD
:109C0000E356CC2253430C4AD1500123E356CC26D1
:109C100073439B180A460146181DFBF7AFFA60789C
:109C2000401C607060780E2800D16570A078401EDE
:109C3000A070E2E73C000020B4010020F8B5044623
:109C4000016880682369E669184363690025334326
:109C50001843724A0B68724E334003430B6021680D
:109C6000486803231B039843E3681843486021684E
:109C7000A069914201D0236A18438B680B263602F3
:109C8000B34303438B606749236867488B420CD119
:109C9000C0688007800F06D0012839D0022835D04F
:109CA000032821D11EE001271FE060498B420AD121
:109CB000C0680C21084027D0042829D0082825D0C6
:109CC0000C2811D10EE093420ED1C168032080020E
:109CD000014019D001208002091A19D0091A15D0A3
:109CE000814201D1082700E010274F4950484039F0
:109CF0008600934232D1002F0CD0022F0DD0042FBA
:109D000010D0082F7FD126E00027EEE70227ECE7EE
:109D10000427EAE7FDF71EFB06E00968C90605D43B
:109D2000304603E0FDF736FB002872D06268510030
:109D30005118814267D81103814264D3010E060293
:109D40005008002330185941FBF7E8F903210902B4
:109D5000411A384A55E00120C003E7E70122E369D0
:109D6000D20393422BD13B0000F0E1F90906090C24
:109D70004D114D4D4D274D00FDF7ECFA09E0FDF773
:109D8000F9FA06E00968C90605D4304603E0FDF794
:109D900001FB00283DD0616840004A088018FBF7AD
:109DA000A7F980B20146244A103991422BD8511CA0
:109DB00001400007400F084329E01046EBE73B0055
:109DC00000F0B5F90906090C2112212121232100F7
:109DD000FDF7C0FA0AE0FDF7CDFA07E00968C90609
:109DE00006D4304604E00EE0FDF7D4FA002810D087
:109DF00061684A081018FBF77BF980B201460E4AE9
:109E00001039914203D9012503E01046F0E721689B
:109E1000C86000206066A0662846F8BD0048004083
:109E2000F369FFEF00380140401002400044004059
:109E300000093D00FFFC0F00EFFF0000F8B50446ED
:109E40004165403000262746028380373E6022204D
:109E5000E0672546206F603500281CD01749C16295
:109E6000216F17480863216F16484863206F866387
:109E7000236F606D9C46134621680246604624317C
:109E8000FCF756FC002806D0102038602E752020E4
:109E9000A0670120F8BD2E7520680168FF220132FD
:109EA00011430160206881680122114381602068AC
:109EB00081684022114381600020F8BD1D9B00088D
:109EC0007B9B0008D19A0008FFB581B005460F467C
:109ED000044660350A9E39E0701C37D0FCF7D0FD8F
:109EE0000499401AB04222D8002E20D02068016880
:109EF00049072BD5C069C043000527D4012021683C
:109F0000C002086220680168FF22A132914301600B
:109F1000206881684908490081602020A067E067C7
:109F20008034206000202875032005B0F0BD206833
:109F30000168FF22A13291430160206881684908CD
:109F4000490081602020A067E067EBE72068C169D5
:109F50003846884305D0002103988142BCD00020B8
:109F6000E3E70121F8E7000010B504491020096873
:109F700008620248FDF700FD10BD000088160020B1
:109F800001490D20887070473C00002010B5FEF795
:109F9000BFFAFEF797FBC82202490348FDF79CFE73
:109FA00010BD0000DC0C002088160020F8B53E4CE7
:109FB000002321783D4A1D46082910D0072947D0A3
:109FC000062950D0052952D0042953D0032954D052
:109FD000002956D0012958D002295AD05BE0A17837
:109FE00000264A1F04E0314FBF5DFB189BB2761C70
:109FF0009642F8DB667927799A195118E3786278E6
:10A00000C9188918C9194018C0430006000E1AD192
:10A01000012E14D0022E16D125482449C018FBF772
:10A02000ADF800F08BFF642000F008FABFF34F8F0B
:10A0300021492048C860BFF34F8F00BFFDE7590892
:10A040001046FFF78FFA2570E570A570A571F8BD71
:10A05000A1795054491CC8B2A071A178491F884207
:10A06000F5D1082001E0607007202070F8BDE07095
:10A070000620FAE760710520F7E7A070E57004207C
:10A08000F3E7552807D10120EFE7AA2803D10220E2
:10A09000EBE7032803D02570E570A570F8BD032019
:10A0A00020702071F8BD00001C0100209A140020CF
:10A0B000A40D00200400FA0500ED00E010B5024AEE
:10A0C000024900F047F910BD79AC00087401002086
:10A0D0002021020C01D010211046020A01D01046A6
:10A0E0000839020901D01046091F820801D0104624
:10A0F000891E420801D0881E7047081A7047F8B5BB
:10A10000040C8BB2264682B25E430D0C1046370C0F
:10A110005843360480190021794116466E43370CA6
:10A1200036048019794126466E438919F8BD30B44A
:10A130007446641E2578641CAB4200D21D46635DE4
:10A140005B00E31830BC18478307FF22DB0E9A4000
:10A150008907090E9940002808DB830809489B00FD
:10A160001B18186890430843186070470007000FD9
:10A170000838830804489B001B18D869904308439B
:10A18000D861704700E400E000ED00E0BFF34F8FBE
:10A1900004490348C860BFF34F8F00BFFDE70000CC
:10A1A0000400FA0500ED00E002E008C8121F08C133
:10A1B000002AFAD170477047002001E001C1121F48
:10A1C000002AFBD1704708B50021684601706B4634
:10A1D000012202212C2000F0EFFC022168460170D0
:10A1E0006B4601222C2000F0E7FC08BD38B5044680
:10A1F0006D20694608706B46012207492E2000F049
:10A20000DBFC0649002C01D0054A00E0054A2E205F
:10A2100000F0B8FC38BD0000060800000618000079
:10A22000070600000716000038B504466B460222F8
:10A230000021362000F08CFBB3212300FFF777FFCD
:10A240000E0F08153A3A3A3A1C273A3A2F34483A50
:10A2500000216846017040784108490014E06946D1
:10A26000087880088000401C04E06946087880086F
:10A270008000801C08701DE0684602780A40483261
:10A2800002704178802001436846417012E06846C0
:10A2900002780A40027040784106490EF4E76946A8
:10A2A00048780221084303E069464878FD210840C8
:10A2B000694648706B4601220021362000F07CFC84
:10A2C000012200AB11463620013300F075FC38BD89
:10A2D00069460878CF21084069462030CAE708B5AA
:10A2E000032168464170012101706B460222002162
:10A2F000362000F061FC0122D20306212D2000F05F
:10A3000041FC012000F09AF80120FFF78DFF08BD05
:10A3100008B5020A69464A7008706B460222042199
:10A320002D2000F049FC0320694608706B4601228D
:10A3300006212D2000F040FC0020694608706B4685
:10A34000012206212D2000F037FC0A212D2000F0EB
:10A35000E5FA08BDF8B516460F460446002503E0A9
:10A360003946B047641C6D1C20780028F8D1284677
:10A37000F8BD0000F8B54A002B4B520DD6182B4AF9
:10A380000C460546142E2BDA002E12DA284BFAF76B
:10A39000C9FF00221346FBF7F5F940D2002C03DA7F
:10A3A0000124E40700253AE02046284337D0214C19
:10A3B00014E0214F0B46F7403B402B4331D01C4B60
:10A3C000FAF7B0FF00221346FBF7DCF927D2002C86
:10A3D00003DD01200005F0400419BC4300251EE008
:10A3E000332E1EDC33460027143BFF43DF40384248
:10A3F00017D00F4BFBF740F800221346FBF7C2F9CA
:10A400000DD2002C0ADD142E0CD03420811B01202B
:10A4100088404019A84200D2641C0546BD4321462D
:10A420002846F8BD641CF9E701FCFFFF9C75008815
:10A430003CE4377E0000F03FFFFF0F007D2110B5A8
:10A44000C900484300F001F810BD002140E000BF02
:10A4500000BF00BF00BF00BF00BF00BF00BF00BF04
:10A4600000BF00BF00BF00BF00BF00BF00BF00BFF4
:10A4700000BF00BF00BF00BF00BF00BF00BF00BFE4
:10A4800000BF00BF00BF00BF00BF00BF00BF00BFD4
:10A4900000BF00BF00BF00BF00BF00BF00BF00BFC4
:10A4A00000BF00BF00BF00BF00BF00BF00BF00BFB4
:10A4B00000BF00BF00BF00BF00BF00BF00BF00BFA4
:10A4C00000BF00BF00BF00BF00BF00BF00BF491CEE
:10A4D0008142BCD370470000FEB5044600200190C5
:10A4E00000906079734940000E5A61782578491EC2
:10A4F0007148CFB20163042D77D0072D75D00021AC
:10A500000291217801736C49E379012292058969EE
:10A51000002B6CD0914381616748217A4173217A85
:10A5200082698907890B0A4382610021042000F0B7
:10A5300034FB324661492E2000F024FB3846FFF7F9
:10A5400055FE5F4E0522705D810040185D4943183D
:10A5500007212B2000F030FB5B49029801220B18E9
:10A560000B21282000F028FB705D584980000A5814
:10A570000C21282000F011FBE0795549800040189B
:10A58000A1794900425A0221272000F0FBFA5148E4
:10A590007E00825B0421272000F0F4FAE079002895
:10A5A00029D0A07804282CD02820694608722022BF
:10A5B0000621272000F0E6FA02AB012226212720FF
:10A5C00000F0FAFA444938014018E178890042580D
:10A5D0000821272000F0E1FAA17A601C627A0902C2
:10A5E000114313D016E000E001E0012188E7114398
:10A5F000F608816190E764220621272000F0C2FA64
:10A60000E0E71020694608720246D1E7334901723B
:10A61000090A4172417A007A0A0202432021272066
:10A6200000F0B0FA2E4F0C2123203A6800F0B5FA62
:10A63000F01982880421232000F0A4FAA0790028D0
:10A640000BD0E0792749012243180021212000F096
:10A65000B3FA03200190012000902A07120F100185
:10A660000243607800218007000B02430198000537
:10A6700002430098400402432079C0064009024387
:10A680006079C00602431F2000F087FAA078617845
:10A690000123084302040848DB030261E17949030E
:10A6A00019430A4302610021082000F076FA0020D5
:10A6B000FEBD000008B0000878010020042800005A
:10A6C000B0AF00080C0000202A000020B8AF00083E
:10A6D000D8AF0008E4AF0008E8AF00084110000060
:10A6E000D0AF00082C00002038B50C4607498A8BF3
:10A6F000002102432C2000F045FA684604706B46A6
:10A70000012206212C2000F057FA38BD78010020E4
:10A7100010B5FFF758FD10BD10B5044604213620D2
:10A7200000F0FCF80121C902002C01D0084300E030
:10A73000884302460421362000F02FFA10BD0000A5
:10A7400038B540206946087000210E2000F0E6F878
:10A750000446002211460E2000F01FFA6B4601222B
:10A7600000210D2000F028FA074A00210F2000F0F8
:10A7700014FA00F0EDF9224600210E2000F00DFA47
:10A7800002480021017338BDF8FF272498010020FA
:10A79000FEB50546042069460870514C00206075DE
:10A7A00021462031206348710873A0836063A06351
:10A7B00000F0C8F84B4E206002E000F0C3F82060C3
:10A7C000B042FAD10020FFF72FFD00F0BBF8464E53
:10A7D00020603078242801D9243806E00621FAF7D1
:10A7E00087FC0622101A40010843020601040A43AE
:10A7F00001020A430243B260706000211E2000F093
:10A80000CCF900F09FF820606B4601220021242043
:10A8100000F0D2F91E20FFF77BFD86B2300AA0734C
:10A820000420FFF775FD074600F08CF8206038061D
:10A83000000E0DD002206946087101AB01221221E1
:10A840002D2000F0B9F9A08B012109030843A08352
:10A8500000F078F820600620FFF75AFD60600720BE
:10A86000FFF756FDA060F006C00E207501D1102044
:10A870002075C0B200F0DCF9E80707D0FFF72FFD24
:10A88000A08B0121C9020843A0830AE005213620DC
:10A8900000F02EF81549084002460521362000F048
:10A8A00071F90120FFF7C0FC0021042000F036F808
:10A8B000A0610021262000F031F81521890308430A
:10A8C00002460021262000F068F9002226213620C9
:10A8D00000F058F900F036F820600020FEBD0000BE
:10A8E000780100203001CADE00000020FFFD0000DA
:10A8F00038B5094C89B280B26B46022200F028F8C4
:10A90000002806D168464078010268460078081899
:10A9100084B2204638BD0000FFFF000038B5002497
:10A92000E44389B280B26B46042200F011F800289B
:10A9300006D103216846435C2202D418491EFAD589
:10A94000204638BD10B500210846FFF7E7FF10BDCF
:10A9500038B5002909D0402420436C462070C8B285
:10A960007F2906D8607002200AE06946087001203D
:10A9700006E0802420436C466070C809A070032064
:10A98000694600F0B5FA38BD10B5144603460A46CC
:10A9900021461120FFF7DCFF10BD10B5034605224C
:10A9A00000211520FFF7D4FF10BD10B50346052286
:10A9B00000211720FFF7CCFF10BD38B50546002059
:10A9C0006946087000F0C4F8FF2401342246002DC7
:10A9D00001D00322120200210D2000F0D3F8002D37
:10A9E00013D06B46012203210F20FFF7B1FF684609
:10A9F0000078000709D5FFF7A3FE224600210D20AD
:10AA000000F0C0F80020C04338BD002038BD10B5AC
:10AA1000024601210A2000F0C0F810BD10B504461E
:10AA200000211A20FFF77AFF000D22030005120B08
:10AA3000024300211A2000F0B0F810BD10B5024604
:10AA400002492E2000F09EF810BD000004180000FE
:10AA5000F8B505466B46012203210420FFF778FF75
:10AA60000126114C3607002D0DD02A4600210C205E
:10AA700000F088F869460878102108436946087094
:10AA8000A069304307E069460878EF21084069462D
:10AA90000870A069B0430B46A06101220321042085
:10AAA00000F08AF8F8BD00007801002010B50246D9
:10AAB0000021182000F066F810BD0000F8B5074628
:10AAC000002568460570B807204C2E4600280ADA93
:10AAD0008020694608706B46012200210D2000F09D
:10AAE0006BF801202073F8076946087821D0062109
:10AAF0000843694608706B46012200210D2000F0D2
:10AB00005BF803210F20FFF7F3FE8121C900084203
:10AB100019D04020694608706B46012200210D20A3
:10AB200000F04AF80020FFF7F7FD00252673ED43FB
:10AB300009E002210843694608706B4601220021A2
:10AB40000D2000F039F82846F8BD000098010020DB
:10AB50001CB56B46012203210F20FFF7F9FE684662
:10AB600000784022C1091040C9014000814208D04C
:10AB7000012069460871024601AB03210D2000F057
:10AB80001BF81CBD08B56B461A70120A5A7089B2C0
:10AB900080B2022200F010F808BD38B500236C46E0
:10ABA000E254120A5B1C042BFADB89B280B2234602
:10ABB000042200F001F838BD38B58024002909D0FE
:10ABC000C02528436D462870C8B27F2907D8687011
:10ABD000022009E0204369460870012004E0204378
:10ABE0006870C809A8700320694600F0BDF938BD37
:10ABF00010B51446012312189B029A4202D9002074
:10AC0000C04310BD0B46821E21460920FFF7D4FF2A
:10AC1000002010BD10B5054A8905126901430A4399
:10AC200000210820FFF7B9FF002010BD78010020A7
:10AC300038B504466B4601220E212B20FFF788FE13
:10AC400068460078E10640094001C90E01436846A4
:10AC500001706B4601220E212B20FFF7ADFF38BD9E
:10AC600010B5002142541C06120A22431B0A491C3B
:10AC70000429F7DB10BD000013B501231A4669460D
:10AC80000248FDF75BF800981CBD00008816002004
:10AC90007CB5002425466846FFF77FFE0420694600
:10ACA000220E2D02154322020C5C1443401EF7D5E0
:10ACB000204629467CBD7CB5002425466846FFF722
:10ACC00074FE04206946220E2D02154322020C5CFC
:10ACD0001443401EF7D5204629467CBDFBF7DEFE17
:10ACE000FEF7E0FCFDF728FC3E493F48002522C066
:10ACF00005608561C5613D490562C1600838FCF7A2
:10AD000063F8FDF705FCFDF7DDFCFDF7B9FCFDF789
:10AD1000CBFB052401222407D1032046FBF7A9FE23
:10AD2000FEF772FAFDF7A8FAFAF756FFFAF724FFD2
:10AD3000FDF786F80721A015FFF7D6FCFFF7E8FC22
:10AD4000012211032046FBF794FE2748C822284918
:10AD5000C830FCF7C1FF274F274E284C3878002811
:10AD60000ED13078002801D0032809D14021244891
:10AD7000FBF772FE002803D101210846FCF738F9E1
:10AD8000E07800282AD06078002827D0E57072B6D5
:10AD900020780F280AD90120194900038861FEF79D
:10ADA000F7FC01201649000388620CE001225103E0
:10ADB0001348FBF75EFEFEF7EBFC0121002249037E
:10ADC0000F48FBF756FE62B6FDF76CF9FAF76AFE1C
:10ADD000A08C0028C2D0401EA084BFE7FDF762F916
:10ADE000BCE70000007C0040C0150020FFFF000011
:10ADF000DC0C0020420000206C0000202401002018
:10AE00000004005010B586B0FDF7E4F91748FBF7D1
:10AE10005EFF14216846FAF7CAF91548009003202E
:10AE2000019000200290052069460007FBF758FDBD
:10AE300069461048FBF754FD69460F48FBF750FD83
:10AE400001210846FCF7D4F8FF2401342046FCF722
:10AE5000A7F80A4908680422104308602046FCF756
:10AE6000AFF8FCF7B5F806B010BD0000C015002023
:10AE7000FFFF000000040050000800500070004078
:10AE800010B50122920216491648FAF729FF144814
:10AE9000154902888A4222D0018014498180FF210D
:10AEA000F531C1800A21018100211E224181D24356
:10AEB00082810122C28181834323C3860287782352
:10AEC00043878287C287024640321184518491842D
:10AED000C183918014238382118200F02FF810BD6A
:10AEE000A40D002000FC0008AA5500003412000048
:10AEF000F0B58C4600251026052109078E620E4C00
:10AF000008E067467F5DE760A768FF07FCD0E76859
:10AF10001F706D1C8542F4DB0020074606E0E760E9
:10AF2000A568ED07FCD0E5681D54401C9042F6D39F
:10AF30008E610020F0BD00000030014070B572B697
:10AF40000124074DA40221462846FAF7AFFE002847
:10AF500004D0224603492846FAF74CFF62B670BD7A
:10AF600000FC0008A40D0020F0B5002510260527E0
:10AF70009C463F070B46BE620C4C06E0595DE16003
:10AF8000A168C907FCD0E1686D1C8542F6DB002092
:10AF900007E06146095CE160A168C907FCD0E1688F
:10AFA000401C9042F5D3BE610020F0BD003001404E
:10AFB0000000010203040005405C0000A05C0400E6
:10AFC000C06C0800805C0400E03F1E00E07D1E00B5
:10AFD00007A9022570889B880A0016000100060058
:10AFE0000100020087008D002D001A3152001A3333
:10AFF0009A001A351D011A376B003B31BE003B33F6
:10B000005E013B3596023B37000099599959EB5147
:10B010008F421E45142E0080EB51F5283333E13A60
:10B02000703DE13AC235852BC2353333C235C23566
:10B03000AE47E13A5138A33051380000000000001B
:10B0400000000102030406070809030406080C10A7
:10B050001820300000000001020304007CB000084A
:10B060000000002078010000C4590008E0B000088A
:10B0700078010020401A0000B8A10008C11307049D
:10B08000380D091E080540082609104008560A1305
:10B090001D043B08BE0516D8BC4010085201033AF7
:10B0A000C842077052030CE5800C1B0202DD140934
:10B0B00001022281F01F6681049889968696798222
:10B0C0001598039814988796749778824397889672
:10B0D0007197778249F1013D294392045220000083
:04000005080050C1DE
:00000001FF
